:100000000C9421010C949E030C943E010C943E012F
:100010000C943E010C943E010C943E010C943E0164
:100020000C943E010C943E010C943E010C943E0154
:100030000C943E010C943E010C943E010C943E0144
:100040000C943E010C943E010C9498020C943E01D9
:100050000C94D1020C943E010C943E010C943E0190
:100060000C943E010C943E010C943E010C943E0114
:100070000C943E010C943E010C94C7020C943E017A
:100080000C943E010C943E010C943E010D09000EAF
:100090007E001551F016212B1A5A281B53A61C411D
:1000A000C41D57221E40F12143A92258292344AFE1
:1000B0002445AE2524F32623F22920202A56CE2BD0
:1000C00046E22C54B82D52B12E25F4314EEC32427A
:1000D0002E3348E73447AC355900365ED9394CC821
:1000E0003A4D3F3B4A2B3C55EA3D26DF3E2AF5413F
:1000F0003CB2424BC94349B3444FCF4529F6462849
:10010000F7493ECC4A3FC04B4CC84C3AAB4D50AD82
:100110004E5F00522200547B00552B005A00005BBA
:100120007D005D7C00613E006608006931316B3402
:10013000346C3737703030712C2E72323273353563
:10014000743636753838792B2B7A33337B2D2D7DE9
:1001500039397C2A2AE000000000000D09000E60F9
:10016000001571E61631E51A7ABC1B73CB1C61BF12
:100170001D77E41E322F2163E12278BB2364A12482
:1001800065DD2534C026335F2920202A76CD2B66F5
:10019000B42C74D02D72BE2E35B6316ED73262D4E7
:1001A0003368E93467E03579D13636D8392CC13A2D
:1001B0006DB73B6A003C75D53D37D63E38A4412C1F
:1001C000C1426B004369C3446FB94530A84639A5A5
:1001D000492EE34A2FBD4B6CCA4C3BC74D70C24EF3
:1001E0002DA2522700545BBA553DAA5A00005B5D10
:1001F000C55D5C00613C006608006931316B3434D8
:100200006C3737703030712C2E7232327335357452
:100210003636753838792B2B7A33337B2D2D7C2A63
:100220002A7D3939E000000000000D0A25303258DF
:1002300020256320000D0A52656164792E2E2E2E32
:10024000000011241FBECFEFD0E1DEBFCDBF11E013
:10025000A0E0B1E0EEE8F0E200E00BBF02C00790E2
:100260000D92A030B107D9F711E0A0E0B1E001C0D4
:100270001D92A032B107E1F70C94B2050C94000076
:10028000CF93C82F8A3019F48DE00E94FB028C2F87
:100290000E94FB02CF910895CF93DF93EC01FC0104
:1002A00021968491882339F00E944001FE01219615
:1002B00084918823C9F7DF91CF9108952F923F92BF
:1002C0004F925F926F927F928F929F92AF92BF9266
:1002D000CF92DF92EF92FF920F931F93CF93DF9312
:1002E000CDB7DEB72C970FB6F894DEBF0FBECDBFEB
:1002F00041E2442E512C4C0E5D1ED201AD90BD90BA
:100300002D01F5010894A11CB11C8491853221F0C6
:10031000882309F4F4C060C03AE0832E912CF501E3
:100320000894A11CB11C84913324232C803311F038
:10033000803281F4282EF5010894A11CB11C84910F
:10034000982F90539A3030F4392EF5010894A11C5F
:10035000B11C849190E08C3611F08C3431F491E032
:10036000F5010894A11CB11C8491282F332728354E
:10037000310509F446C0293531059CF42434310592
:1003800009F443C02534310524F423343105F1F058
:1003900023C02335310519F12535310509F45BC03A
:1003A0001BC023373105D9F0243731053CF42336FF
:1003B000310561F02436310541F10EC02537310594
:1003C00009F449C028373105E1F006C0F20182E0A6
:1003D00090E0480E591E80810E94400192CFF201A8
:1003E000A2E0B0E04A0E5B1EC080D180F6018081A1
:1003F000882309F486CFD6018D916D010E944001BA
:10040000F5CF20E1822E912C26C0992351F0F201E4
:1004100084E090E0480E591EE080F1800281138153
:100420000CC0F201A2E0B0E04A0E5B1E8081918117
:100430007C010027F7FC0095102F17FF22C01095B4
:100440000095F094E094E11CF11C011D111D8DE25A
:100450000E94400116C0992351F0F20184E090E01F
:10046000480E591EE080F180028113810AC0F2011A
:10047000A2E0B0E04A0E5B1E808191817C010027E2
:1004800011278CE0C82ED12CCC0EDD1E1C86C40199
:10049000AA27BB273C014D01C801B701A401930164
:1004A0000E94EF0F262F205D2A330CF0295FD60122
:1004B0002E936D01C801B701A40193010E94EF0FB3
:1004C00079018A0131103A94E114F1040105110512
:1004D00019F73A94BFEF3B1639F0F60122926F01FB
:1004E0003A94FFEF3F16C9F7D6018C91882309F49F
:1004F00008CFF60181916F010E944001F5CF2C9643
:100500000FB6F894DEBF0FBECDBFDF91CF911F9124
:100510000F91FF90EF90DF90CF90BF90AF909F90A2
:100520008F907F906F905F904F903F902F900895A5
:100530001F920F920FB60F9211242F938F939F93B8
:10054000EF93FF938CB1809302018091140180316D
:10055000A0F48091150120911401820F912D911D1D
:10056000FC012F5F20931401807F9370E81BF90B2F
:10057000EC5FFE4F809102018083FF91EF919F918C
:100580008F912F910F900FBE0F901F9018951F9273
:100590000F920FB60F9211240F900FBE0F901F9065
:1005A00018951F920F920FB60F9211245398109224
:1005B00003010F900FBE0F901F90189580911401AA
:1005C0008823E1F3539880911401815080931401A2
:1005D00080911501E82FFF27EC5FFE4F8F5F80931E
:1005E0001501E08180911501803110F01092150104
:1005F0008E2F99270895982F809103018130E1F380
:10060000539A9CB981E08093030108950F931F933F
:10061000CF93FC01C1918F01CC2371F0CA3019F442
:100620008DE00E94FB028C2F0E94FB02F801819159
:100630008F01C82F882391F7CF911F910F910895B3
:100640001F93CF93DF93EC01FC01219614911123AA
:1006500071F01A3019F48DE00E94FB02812F0E9484
:10066000FB02FE0121968491182F882391F7DF91D8
:10067000CF911F91089510921501809115018093DB
:10068000140110920301119A199A88E58AB986E03B
:100690008093950057981092900087E689B9089545
:1006A000CF93C82F82958F708A3010F4805D01C07F
:1006B000895C0E94FB028C2F8F708A3010F4805D61
:1006C00001C0895C0E94FB02CF910895982F10927F
:1006D0009B0088E180939A0086E080939D001092B1
:1006E00098009093990080919A00806880939A0076
:1006F000089580919B008823E4F780919C009927BE
:1007000087FD90950895982F80919B0085FFFCCFE1
:1007100090939C000895CF93DF93EC018881882308
:1007200051F089910E94830380E090E00197F1F7F6
:1007300088818823B1F7DF91CF9108951F920F929E
:100740000FB60F9211248F938091180180688093C7
:1007500018018F910F900FBE0F901F9018958091E8
:100760006A00826080936A0089B7816089BF0895BA
:1007700010921D0190911E01906490931E01809330
:100780001A0110921601909AE0E0F0E0CF01019773
:10079000F1F7919A81B3836081BB80E08A95F1F78C
:1007A00090983197F1F79198889885E08A95F1F7BC
:1007B000089510921B0180911E01282F332724FFDA
:1007C00003C084E080931B0123FF05C080911B01BF
:1007D000826080931B0125FF05C080911B01816011
:1007E00080931B010895CF93482FC0E0803EF1F025
:1007F000803F21F481E08093010118C080910101C4
:100800008130B9F4C093010180E090E0423111F4ED
:1008100081E090E020E030E0493511F421E030E063
:10082000822B932B892B11F0C093000180E090E084
:1008300011C1642F77276935710501F16A3571059A
:100840007CF462317105D1F0633171052CF46E30A6
:10085000710509F43FC04BC06835710539F147C0D7
:100860006E37710579F06F37710524F467377105BC
:1008700089F03DC06A3F710541F139C081E0809344
:100880000001E6C080911E0185FF02C08F7D09C076
:10089000806207C080911E0183FF02C0877F01C074
:1008A000886080931E010E94D9030DC080911E01B3
:1008B00084FF02C08F7E01C0806180931E010E9470
:1008C000D90310921F018DEE02C080911B010E947E
:1008D000B803BEC080911901882321F481E0809380
:1008E000190102C0C093190110921F01B1C080917B
:1008F0001F01882309F098C0E091000190911E012A
:10090000EE2309F04AC094FD24C09E2F23E0EBE5BE
:10091000F1E008C0882349F09F5F929FF001112405
:10092000E55AFE4F84918417A9F783E0989F9001C0
:100930001124F901E55AFE4F8491841709F074C01F
:1009400080911901F901E80FF11DE45AFE4FC4919D
:100950006BC09E2F23E0ECE8F0E008C0882349F04C
:100960009F5F929FF0011124E457FF4F84918417F9
:10097000A9F783E0989F90011124F901E457FF4FF4
:100980008491841709F050C080911901F901E80F92
:10099000F11DE357FF4FC49147C094FD23C0982F2A
:1009A00023E0ECE8F0E008C0882349F09F5F929FC5
:1009B000F0011124E457FF4F84918417A9F783E0D5
:1009C000989F90011124F901E457FF4F84918417F7
:1009D00059F580911901F901E80FF11DE357FF4F17
:1009E000C49122C0982F23E0EBE5F1E008C08823F2
:1009F00049F09F5F929FF0011124E55AFE4F8491C8
:100A00008417A9F783E0989F90011124F901E55A12
:100A1000FE4F8491841741F480911901F901E80F88
:100A2000F11DE45AFE4FC4918C2F99279F938F9309
:100A30007F936F938AE292E09F938F930E945E016F
:100A40008DB79EB706960FB6F8949EBF0FBE8DBFAA
:100A50008C2F9927CF91089530E020911E0180912D
:100A60001D0126FF37C08F5F80931D0199278930B4
:100A7000910549F089309105C4F08A30910549F01B
:100A80000B9749F012C080911601882311F09198BC
:100A900046C0919A44C0919889982F7B20931E015B
:100AA00030931D01309316013AC080911D018823B7
:100AB000B1F120911A0120FF08C0919A809116018E
:100AC00091E089278093160101C091982695209383
:100AD0001A0125C0982F9F5F90931D018150883087
:100AE00058F480911701869580931701819B17C058
:100AF00080688093170113C09B3088F080911701A4
:100B0000803E31F480911F018F5F80931F0105C0EB
:100B10000E94F303382F10921F0110921D01832FA2
:100B20009927089581B38C7F81BB82B3836082BB98
:100B3000109218010E94AF0310921E01109217012B
:100B400010921D011092190110921C018091180140
:100B500087FFFCCF0E942C05809118018F7780932E
:100B60001801F4CFCFEFD0E1DEBFCDBF0E943B0331
:100B7000789485E392E09F938F930E945E010E9498
:100B800092050F900F90FFCF2F923F924F925F925E
:100B90006F927F928F929F92AF92BF92CF92DF928D
:100BA000EF92FF920F931F93CF93DF93CDB7DEB7F2
:100BB0002A970FB6F894DEBF0FBECDBF1C015A01B5
:100BC0006B012D831F830E8327FF02C01D8205C08A
:100BD0002D81263214F065E26D8318862101C10152
:100BE00088969A87898720E030E040E050E0C6018F
:100BF000B5010E94760E88235CF4EE81FF8180812E
:100C00009181826091838083D7FAD094D7F8D09471
:100C1000AE014F5F5F4FC601B5010E94D60E5B016A
:100C20006C0189819A81AB81BC8120E030E040E099
:100C300050E0BC01CD010E94760E882309F44AC021
:100C400009851A852AC02DEC3CEC4CEC5DE3C4010F
:100C5000B3010E94060FDC01CB01AE014F5F5F4F75
:100C6000BC01CD010E94D60EDC01CB012AE939E995
:100C700041E251E4BC01CD010E94060FDC01CB0131
:100C8000BC01CD010E945B0EDC01CB01805DF8014F
:100C900082938F01F885FF5FF88769807A808B8067
:100CA0009C8020E030E040E050E0C401B3010E94AD
:100CB000760E882319F02016310628F289859A8548
:100CC0000817190768F5F80181918F01F2018193E6
:100CD0002F01F4CF20E030E040E050E0C601B50144
:100CE0000E94790E1816E4F405C057016801988532
:100CF0009150988720E030E040E251E4C601B50110
:100D00000E94060F7B018C0120E030E040E85FE3A9
:100D10000E94760E87FDE9CFE982FA820B831C835D
:100D2000EE81FF814081518153FF15C0F885FD3F61
:100D300094F02F2F332727FD30956D81862F99272B
:100D400087FD90950196281739072CF45460EE81A1
:100D5000FF8151834083EE81FF81808191819C01DD
:100D60002070347092FD03C0FD81FF5FFD836D81B3
:100D7000062F112707FD1095020D131D232B39F0A7
:100D8000E8858E2F992787FD9095080F191F02156A
:100D9000130520F5F10158C089859A854816590632
:100DA00000F520E030E040E251E4C601B5010E94C8
:100DB000060FAE014F5F5F4F0E94D60E5B016C01C4
:100DC00089819A81AB81BC81BC01CD010E945B0EFF
:100DD000DC01CB01805DF20181932F010415150523
:100DE000D8F6E985FA850E171F0718F0F10117A24A
:100DF0002CC02801F80180818B5F80838A331CF12D
:100E000020E331E3F80120832016310628F4829193
:100E10008F018F5F808313C0F8013083F885FF5FF7
:100E2000F887EE81FF818081918192FF08C02414B0
:100E3000350410F4F20120830894411C511CF80180
:100E400080818A33FCF6F2011082F8858F2F992772
:100E500087FD90952A960FB6F894DEBF0FBECDBFE2
:100E6000DF91CF911F910F91FF90EF90DF90CF9086
:100E7000BF90AF909F908F907F906F905F904F90BA
:100E80003F902F9008952F923F924F925F926F92D2
:100E90007F928F929F92AF92BF92CF92DF92EF920A
:100EA000FF920F931F93CF93DF93CDB7DEB7EE97EB
:100EB0000FB6F894DEBF0FBECDBF8824992454012D
:100EC0003C0178AF6FAB1A011EAA1DAAFC01178264
:100ED0001682838181FD1EC48FEF9FEF2EC48FA9E0
:100EE00098AD019698AF8FAB6DA97EA960FFFEC348
:100EF00089AD80538A30C8F499AD903331F45520D0
:100F000021F463FD02C07160ABC18AE0589E502C91
:100F10001124E9AD5E0EF0ED5F0E57FE02C05FE7F3
:100F2000552E63FDF7C3452CF5C329AD25562EAFCD
:100F3000233028F089AD8554833008F01EC1F101BB
:100F400084E090E0280E391EE080F1800281138158
:100F50004701580163FD02C046E0542E37EBC32E13
:100F60003FEFD32EC622D722DEAACDAAC801B701F1
:100F70000E94C60E892BB9F08EE48B83898381E4AD
:100F80008A83FE013496FCAFEBAFFEADF33008F080
:100F9000ADC28981805E89838A81805E8A838B81EC
:100FA000805E8B83A3C2C801B7010E94CD0E892B3E
:100FB000C9F089E48B838EE48A8386E48983CE0139
:100FC00004969CAF8BAF20E030E040E050E0C801D9
:100FD000B7010E94760E8823C4F68DE28C83FE0151
:100FE0003596D1CF80E092E0C82AD92ADEAACDAAD0
:100FF000E9AD8E2F992787FD90958734910509F4E7
:101000005CC0883491053CF48534910599F08634B0
:10101000910561F17FC38636910541F187369105CF
:1010200024F48536910531F075C38736910509F4AE
:1010300044C070C38E010B5C1F4F252DB501A40168
:10104000CE010D960E94C4058DAFFCEF4F0E151416
:101050000CF44A94CE010D969CAF8BAFFC0101902D
:101060000020E9F731978E2E881ABFC18DA99EA95D
:1010700094609EAB8DAB8E010B5C1F4F252DB5018F
:10108000A401CE010D960E94C4058DAF15140CF479
:101090004A94FE013D96FCAFEBAFFDAD1F1654F434
:1010A000EBADFCAD01900020E9F731978E2E2BAD12
:1010B000821A9BC1852C839498C18DA99EA99860A2
:1010C0009EAB8DAB252D552009F421E08E010B5CE4
:1010D0001F4FB501A401CE010D960E94C4058DAF2E
:1010E0008DA99EA992FF27C08DAD850D8150882EB8
:1010F00087FD15C08DAD881694F09E012F5F3F4F80
:10110000E82DFF27E7FDF095E20FF31F848580337C
:1011100031F48A9487FC03C09DAD89168CF787FC57
:1011200003C0EDAD8E1614F4552418C0582CFDAD37
:101130005F1A539413C0852C15147CF49E012F5F05
:101140003F4FE82DFF27E7FDF095E20FF31F848561
:10115000803319F48A941814A4F3582CE82DFF272F
:10116000E7FDF095EC0FFD1F16868DA99EA992FD57
:101170008DCF29AD225029AF68CF63FF04C0552021
:1011800011F421E0522EE9AD8E2F992787FD90951D
:101190008936910509F4A5C08A3691057CF5833519
:1011A000910509F483C084359105BCF48B32910517
:1011B00009F443C08C3291054CF48032910509F456
:1011C0003FC08332910509F443C08AC28D32910534
:1011D000E9F18E329105F1F183C28336910509F46C
:1011E00042C0843691052CF48835910509F4AEC0CF
:1011F00077C28436910509F474C072C280379105B4
:1012000009F49FC08137910544F48C36910539F17A
:101210008F36910509F492C063C28537910509F4B0
:1012200097C08637910524F48337910521F158C280
:101230008837910509F48AC053C260617EAB6DABFB
:101240008DA99EA980629EAB8DAB64C2606808C008
:10125000606406C068607EAB6DAB55245BC26460A1
:101260007EAB6DAB57C2F10182E090E0280E391ED3
:1012700080804A943BC1F10182E090E0280E391E43
:10128000A081B1814D0163FF09C0852D992787FD9C
:101290009095BC01CD010E94C40D1FC0FD010190BD
:1012A0000020E9F73197EA1BEAAF18C0F10182E0AC
:1012B00090E0280E391E0190F081E02D4F0163FF70
:1012C00009C0852D992787FD9095BC01CF010E940B
:1012D000B90D03C0CF010E94B00D8AAF9AAD491A73
:1012E00005C162FF0AC0F10184E090E0280E391EBA
:1012F00020813181428153810CC0F10182E090E074
:10130000280E391E808191819C01442737FD40952C
:10131000542F49015A0157FF0BC062607EAB6DAB81
:10132000B094A09490948094811C911CA11CB11C39
:101330008DA99EA98F7B9EAB8DAB27C098E09AAFFD
:1013400007C060647EAB6DABE8E7E9AFF0E1FAAFF0
:101350006DA97EA962FF0AC0F10184E090E0280E29
:10136000391E20813181428153810AC0F10182E01E
:1013700090E0280E391E808191819C0144275527D9
:1013800049015A016F7C7EAB6DABFE013196FCAF1B
:10139000EBAF6F01FAADEF2EFF2400271127C50137
:1013A000B401A80197010E94EF0FDC01CB01EBAD66
:1013B000FCAD80838A3024F0F9AD8F0F815201C0DB
:1013C000805DEBADFCAD8193FCAFEBAFC501B4012B
:1013D000A80197010E94EF0F49015A01211531051B
:1013E00041055105E1F68BAC8C184DA95EA9CA01E7
:1013F00082739070892B09F04A9446FF0DC0842DAA
:10140000992787FD9095FAADF03121F49EEF492E92
:10141000480E02C0482E4A9443FF0EC0252D3327A4
:1014200027FD3095882D99278217930724F0477F51
:101430005EAB4DAB01C058188DA99EA983FF02C0B9
:10144000451801C0481880789170892B51F4842D7B
:101450004A94181634F4B30180E290E00E94120E10
:10146000F6CF8DA99EA981FF04C0B3018DE290E063
:101470000BC084FF04C0B3018BE290E005C085FF80
:1014800005C0B30180E290E00E94120E8DA99EA9D2
:1014900086FF10C0B30180E390E00E94120E2AADD7
:1014A000203141F4B301E9AD8E2F992787FD909546
:1014B0000E94120E8DA99EA990FF0AC0842D4A9405
:1014C000181634F4B30180E390E00E94120EF6CFB8
:1014D0008DA99EA983FF0AC0852D5A94181634F44D
:1014E000B30180E390E00E94120EF6CF8DA987FD34
:1014F0000AC0842D4A94181634F4B30180E290E0B7
:101500000E94120EF6CFF9ADF33631F4882DB301F7
:10151000992787FD9095C0C029AD2337B9F48AADCE
:1015200081508AAF8F3F09F4CEC0F40180810894C6
:10153000811C911CB301992787FD90950E94120E82
:101540009AAD91509AAF9F3F81F7BDC0E9ADE335A9
:1015500081F4FAADF150FAAFFF3F09F4B4C0F401E1
:101560008491B30199270E94120E0894811C911C4A
:10157000F0CF8DA99EA991FF92C092FF1DC02DAD05
:101580001216B4F421502DAF2F3F81F0EBADFCAD1E
:101590008191FCAFEBAFB301992787FD90950E9435
:1015A000120EFDADF150FDAFFF3F81F71DAE0FC034
:1015B000B30180E390E009C0EBADFCAD8191FCAFDD
:1015C000EBAFB301992787FD90950E94120E151479
:1015D0002CF4B3018EE290E00E94120E8DA99EA918
:1015E00092FF20C08DADF82FFF5FFDAF0DC0852DA0
:1015F0005A941816BCF4B30180E390E00E94120ED6
:101600008DAD282F2F5F2DAF88238CF30BC0852D38
:101610005A9418167CF4882DB301992787FD90956C
:101620000E94120EEBADFCAD8191FCAFEBAF882EAA
:10163000882369F78DA99EA992FD45C0B301F9AD34
:101640008F2F992787FD90950E94120E2DAD215066
:101650002DAF27FF09C0B3018DE290E00E94120E6A
:101660008DAD81958DAF05C0B3018BE290E00E94F6
:10167000120E6AE070E0EDAD8E2F992787FD9095F0
:101680000E94DC0F4B015C01B301C401C0960E94B3
:10169000120EB301C501C0960E94120E14C08E0135
:1016A0000F5F1F4F8BAD9CAD8017910761F0EBADC5
:1016B000FCAD8291FCAFEBAFB301992787FD90950C
:1016C0000E94120EEFCF8DA987FF0DC0842D4A9482
:1016D00018164CF4B30180E290E00E94120EF6CF8F
:1016E000B3010E94120E1EAA1DAA14C099AD953214
:1016F00049F481E090E09EAB8DAB5524452CEAE0A7
:10170000EAAF08C0B301F9AD8F2F992787FD9095F7
:101710000E94120EF301838183FF04C0EFA9F8AD8C
:10172000F49103C0EFA9F8ADF081F9AF29AD222300
:1017300009F0D5CBF30186819781EE960FB6F89428
:10174000DEBF0FBECDBFDF91CF911F910F91FF90F4
:10175000EF90DF90CF90BF90AF909F908F907F9051
:101760006F905F904F903F902F9008952F923F92EF
:101770004F925F926F927F928F929F92AF92BF92A1
:10178000CF92DF92EF92FF920F931F93CF93DF934D
:10179000CDB7DEB727970FB6F894DEBF0FBECDBF2B
:1017A0005C011B014A0166244424552462012FEF89
:1017B0003FEF3B832A83FC01578246825D824C8245
:1017C000838180FD8DC1C901B2C10894211C311CE7
:1017D00060FE79C1F5E27F1619F42EEF622280C116
:1017E000872D992787FD90950E943410782E282FF9
:1017F000332727FD30952C36310579F12D3631050B
:10180000A4F42436310509F47CC02536310524F4CE
:101810002336310529F13FC12836310509F460C16D
:101820002936310509F46DC036C123373105A9F1D8
:10183000243731054CF42F36310509F459C02037CF
:10184000310509F45AC027C12537310509F457C0BD
:101850002837310509F451C01EC134E0632A40C164
:10186000F40182E090E0880E991E0190F081E02D55
:10187000FF83EE83C5010E94CF0D6C019FEFC91657
:101880009FEFD90609F438C1EE81FF81C08203C100
:10189000B501C6010E943F0E28C0F40122E030E0ED
:1018A000820E931EE080F180C5010E94CF0D6C0175
:1018B0000E942510892BC1F73FEFC3163FEFD306D7
:1018C00009F41AC1C6010E942510892B09F7F701F6
:1018D000C0820894E11CF11CC5010E94CF0D6C016F
:1018E0008FEFC8168FEFD80669F7F7011082D3C0C3
:1018F00098E09983E2E06E2A04C0F0E1F98322E0E7
:10190000622AC5010E94CF0D6C010E942510892B0F
:10191000C1F73FEFC3163FEFD30609F4EDC08DE2E8
:10192000C81619F09BE2C91669F4EDE2CE1611F45F
:10193000F8E06F2AC5010E94CF0D6C018F5F9F4FA9
:1019400009F4DAC030E3C31679F5EE24FF248701E9
:10195000C5010E94CF0D6C018FEFC8168FEFD8061E
:1019600009F46FC0C6010E9434108837C1F49FE6A5
:10197000791631F0E4E67E1619F0F5E77F1629F4C2
:10198000B501C6010E943F0E5CC020E12983C5015C
:101990000E94CF0D6C018F5F9F4F31F452C089E6DA
:1019A000781611F498E09983EE24FF248701C6018C
:1019B0000E943410C0979F838E838A30910544F033
:1019C000C1979F838E8397FD03C00A969F838E8362
:1019D000EE81FF81F7FD08C0F9818F2F99272E81B5
:1019E0003F81281739072CF0B501C6010E943F0E30
:1019F0001EC08981282F332744275527C801B701E6
:101A00000E94BD0F7B018C01EE81FF81CF01AA27CF
:101A100097FDA095BA2FE80EF91E0A1F1B1FC501DE
:101A20000E94CF0D6C018F5F9F4F09F0C0CF63FE06
:101A300008C010950095F094E094E11CF11C011D84
:101A4000111D262D3327C90186709070069731F439
:101A5000F40122E030E0820E931E0EC021FF06C08A
:101A6000F40182E090E0880E991E10C0C401029635
:101A700022FF0AC0F4014C010190F081E02DE082C8
:101A8000F1820283138307C0F4014C010190F081BD
:101A9000E02DF182E082F501868197812C813D81E4
:101AA0002817390734F40894411C511C1B821A82F0
:101AB00008C03EE6731601F58FEFC8168FEFD80603
:101AC000D9F066240DC095E2791651F481E0682EB4
:101AD000EAE0E983F5010680F781E02DFD83EC83E0
:101AE000F501838183FF03C0F101749002C0F1010D
:101AF0007080772009F069CE60FE0DC0F501868107
:101B000097812C813D81281739072CF40894411CBA
:101B1000511C1B821A823FEFC3163FEFD30631F4EC
:101B20004114510419F48A819B8101C0C201279696
:101B30000FB6F894DEBF0FBECDBFDF91CF911F91DE
:101B40000F91FF90EF90DF90CF90BF90AF909F905C
:101B50008F907F906F905F904F903F902F9008955F
:101B6000FC0105900020E9F7809590958E0F9F1F4E
:101B70000895FC010590615070400110D8F78095E0
:101B800090958E0F9F1F0895FC0161507040019049
:101B90000110D8F7809590958E0F9F1F0895CF93D1
:101BA000DF93EC014B81842F992780FF2EC086FFA5
:101BB00009C04F7B4B838E819F8101969F838E83CB
:101BC0008A812CC082FF11C0E881F9818081282F91
:101BD000332727FD30952115310519F440624B83D9
:101BE00014C03196F983E88313C0EA85FB85CE01E2
:101BF00009959C0197FF0CC08B8199272F5F3F4F60
:101C000011F4806101C080628B838FEF9FEF07C06A
:101C10008E819F8101969F838E83822F9927DF91EA
:101C2000CF9108950F931F93CF93DF938C01EB0116
:101C30008B81992781FF1CC082FF0DC02E813F81BF
:101C40008C819D812817390764F4E881F98101931B
:101C5000F983E88306C0E885F985802F0995892BEB
:101C600039F48E819F8101969F838E83C80102C0C3
:101C70008FEF9FEFDF91CF911F910F910895AC01EE
:101C8000FB012381822F992780FF06C086FD04C0B7
:101C90008FEF4F3F580719F48FEF9FEF089542835E
:101CA00020642F7D23838681978101979783868384
:101CB000842F9927089597FB47D09F3738F0FEE986
:101CC000F91B982F872F762F6B2F05C05AC096953A
:101CD000879577956795F150D0F73EF4909580956C
:101CE000709561957F4F8F4F9F4F08950ED05EF096
:101CF00004C00BD026F001C008D019F020F48FEFFB
:101D0000089580E0089581E0089597FB092E052647
:101D100000F8689410D0E89407FC07C062177307B6
:101D20008407950721F008F4009407949894089587
:101D3000052E092607FA440F551F5F3F79F0AA27A1
:101D4000A51708F051E04795880F991F9F3F31F084
:101D5000BB27B91708F091E0879508959F919F914F
:101D6000112408C197FB880F991F9F3F31F0BB27B3
:101D7000B91708F091E0879508959F919F911124DC
:101D8000F9C0662777278827992708959F3F59F438
:101D9000803C49F481E0992708959068892387233E
:101DA00086238395B9F3882799270895DBDFCF939E
:101DB000DF93D52FC42F5527442733272227992374
:101DC000D9F09F37C8F0F92FBDD0592F482F372FA2
:101DD000262FF63968F46FDFA6D0C030CD0721F08A
:101DE00069937993899399939058DF91CF9157C0D4
:101DF0009927882777276627C030CD0721F02993B8
:101E0000399349935993DF91CF919CC091DF01D0D1
:101E100099C0992339F0552329F09F575F57950FA3
:101E200013F49AF1B1CF91589F3FE1F3629FA12D36
:101E30000F92BB27639FA00DB11DEE27729FA00DCF
:101E4000B11DEE1FAF93AA27649FB00DE11D739FD4
:101E5000B00DE11DAA1F6627829FB00DE11DA61FD0
:101E60005527749FE00DA11D551F839FE00DA11DF7
:101E7000561F849FA00D511D852F7A2F6E2F1F9006
:101E80000F9088231AF4939539F474C0000C111C38
:101E9000BB1F661F771F881F012808955058192EF1
:101EA00047DF01D04FC0BA17620773078407950751
:101EB000B1F188F40EF410940B2EBA2FA02D062E3B
:101EC000622F202D072E732F302D082E842F402DAA
:101ED000092E952F502DFF275523B9F0591B49F096
:101EE000573E98F0469537952795A795F04053951E
:101EF000C9F776F0BA0F621F731F841F30F48795FD
:101F000077956795B795F040939517FA0F2E08953A
:101F1000BF1BBB27BA0B620B730B840BF6CFDEF62D
:101F200033CFE89403C097FB0EF4D8DEB62F672FAB
:101F3000782F892F9EE9002405C09A95BB0F661F54
:101F4000771F881F11249923A1F08823B2F79F3FA0
:101F500059F0BB0F48F421F4002011F460FF04C0D5
:101F60006F5F7F4F8F4F9F4F881F9795879597F98A
:101F7000089507CF9FEF80EC0895629FD001739F73
:101F8000F001829FE00DF11D649FE00DF11D929F15
:101F9000F00D839FF00D749FF00D659FF00D992754
:101FA000729FB00DE11DF91F639FB00DE11DF91F78
:101FB000BD01CF011124089597FB092E07260AD0F1
:101FC00077FD04D02ED006D000201AF470956195CC
:101FD0007F4F0895F6F7909581959F4F0895A1E260
:101FE0001A2EAA1BBB1BFD010DC0AA1FBB1FEE1F93
:101FF000FF1FA217B307E407F50720F0A21BB30BDE
:10200000E40BF50B661F771F881F991F1A9469F759
:1020100060957095809590959B01AC01BD01CF01B5
:102020000895AA1BBB1B51E107C0AA1FBB1FA6171F
:10203000B70710F0A61BB70B881F991F5A95A9F771
:1020400080959095BC01CD010895911113C0803207
:1020500051F08A3041F08C3031F08D3021F08930F0
:1020600011F08B3099F708958F9309D08F9109F073
:102070008062089599278827089585FDFBCF8062A7
:0E2080009111F8CF8136ECF38B37DCF7089521
:00000001FF
